:100000000C94BB020C9402030C9402030C940203A4
:100010000C9402030C9402030C9402030C9402034C
:100020000C9402030C9402030C94D20C0C94A40DB7
:100030000C9402030C9402030C9402030C9402032C
:100040000C9402030C9470220C9402030C9402038F
:100050000C9402030C94001C0C9402030C940203F5
:100060000C9402030C9402030C9402030C940203FC
:100070000C9402030C9402030C9402030C940203EC
:100080000C9402030C9402030C9402030C940203DC
:100090000C9402030C9402030C9402030C940203CC
:1000A0000C9402030C9402030C940203110E330E01
:1000B000210F330E210F780E9B0E210FF00E030F30
:1000C000EF11EF112C122C126F12AD12C614C614C0
:1000D000C612C614C713C7139A14C614C614B11493
:1000E0000000F0A1F0A2F0A335812B77297FE10079
:1000F000E00000001E00140004831D83E2004D0098
:100100001F001A0016001B00E3004C00200008002E
:100110000700060050002A00210015000900190000
:100120004F004A00220017000A0005000000E0000E
:100130002C082B0200002B000000E3002D00C30060
:100140000000E3040000E20023001C000B0011008B
:100150000000E302240018000D00100052004B00C4
:1001600025000C000E00360051002C002600120065
:100170000F0037002F002800270013003382388239
:1001800030004E002E003177347FE500C1000000C2
:100190000100010001000100010000003A001E0200
:1001A00020022202010001003B001F022102230263
:1001B000010001003C002F0226022F000100010077
:1001C0003D00300227023000010001003E003102F4
:1001D0003500350200000100010036020000690010
:1001E000000001000100370200006A000000010069
:1001F0003F003302330024020000010040002400CD
:1002000021001E00270001004100250022001F00E0
:100210003700010042002600230020002E000100CC
:100220004300310025022D002E020100440045004C
:10023000460028000100000001000100010001004B
:100240000100000001000100010001000100AA00FE
:1002500001000100010001000100A80001000100EF
:10026000010001000100AE000100010001000100D9
:100270000100A90001000100010001000000AC0024
:1002800001000100000001000000AB0001000100BE
:10029000000001000000AC000100010001000100AD
:1002A0000000AB0001000100010001000100A900F5
:1002B00001000100010001000100AE000100010089
:1002C000010001000100A80001000100010001007F
:1002D0000100AA000100010001000100010000006E
:1002E000A600010001000100010000000100010062
:1002F000010001000100010001000100F200010005
:10030000010001000100F000F10001000100010006
:1003100001000100F30001000100010001000100E3
:10032000F400F50000000100A5000100000001003C
:1003300000000100010001000000010000000100B8
:100340000100010050000100000001000100010057
:1003500051000100010001000100010052000100F4
:1003600001000100010001004F0001000100010037
:100370000100010001000100010001000100010075
:100380000100010001000000160345007200670033
:100390006F0044006F007800200045005A00000004
:1003A00016034500720067006F0044006F0078007C
:1003B000200045005A0000000403090409026D00F2
:1003C000040100A0FA090400000103010100092151
:1003D00011010001223F000705810308000A0904FA
:1003E00001000103010200092111010001224D0059
:1003F0000705820308000A09040200010300000047
:100400000921110100012236000705830308000AB3
:100410000904030001030000000921110100012269
:1004200039000705840310000112011001000000CB
:1004300008EDFE071301000102000105010906A1F4
:1004400001050719E029E7150025019508750181C7
:100450000205081901290595057501910295017597
:100460000391010507190029771500250195787575
:10047000018102C005010980A10185021601002643
:10048000B7001A01002AB700751095018100C00558
:100490000C0901A1018503160100269C021A010026
:1004A0002A9C02751095018100C005010902A10175
:1004B0000901A10005091901290515002501950566
:1004C000750181029501750381010501093009312A
:1004D0001581257F95027508810609381581257FCC
:1004E000950175088106050C0A38021581257F954E
:1004F0000175088106C0C005010906A1010507199B
:10050000E029E7150025019508750181029501751F
:1005100008810105081901290595057501910295C4
:1005200001750391010507190029FF150025FF95A5
:100530000675088100C000000000000000000000F7
:1005400000010204060A0F17202C3A4A5D71879DAC
:10055000B3C7DAE9F5FCFFFCF5E9DAC7B39D8771AB
:100560005D4A3A2C20170F0A060402010000000021
:1005700000000000000011241FBECFEFDAE0DEBF54
:10058000CDBF04B603FE27C08091EE019091EF012C
:10059000A091F001B091F1018730904BA740B04B92
:1005A000D1F41092EE011092EF011092F00110922E
:1005B000F10114BE84B7877F84BF0FB6F894A89565
:1005C00080916000886180936000109260000FBE8F
:1005D000E0E0FFE3099511E0A0E0B1E0ECE8F8E429
:1005E00002C005900D92A433B107D9F721E0A4E32E
:1005F000B1E001C01D92AE3EB207E1F70E94130ABE
:100600000C9444240C94000061110BC0FC01828105
:10061000882321F085EE0E94831003C085EE0E949E
:100620004B1180E090E0089508956091B1017091C0
:10063000B2018091B3019091B4010E94291B569898
:100640005E9825982D9826982E9827982F98823076
:1006500039F0833041F0813041F4259A2D9A089584
:10066000269A2E9A0895279A2F9A08950C94150386
:1006700056985E9825982D9826982E9827982F980A
:100680008FEF90E0909389008093880090938B0087
:1006900080938A0090938D0080938C00259A2D9AE8
:1006A0002FEF80E792E0215080409040E1F700C0BA
:1006B0000000269A2E9A2FEF80E792E0215080408A
:1006C0009040E1F700C00000279A2F9A2FEF80E7B3
:1006D00092E0215080409040E1F700C00000259852
:1006E0002D982FEF80E792E0215080409040E1F775
:1006F00000C0000026982E982FEF80E792E021504E
:1007000080409040E1F700C0000027982F9856984D
:100710005E9825982D9826982E9827982F980895BA
:1007200089EA8093800089E08093810024982C9846
:100730003F988AB18F748AB96E98479A8BB1806B53
:100740008BB9769A0E9438030C94140380E280934C
:1007500000018091340181110EC00E94F50381E0F7
:10076000809334012FEF83ED90E32150804090403F
:10077000E1F700C0000080E40E94FB0380930001C9
:1007800081112EC00E94250480930001811128C090
:100790000E94250480930001811122C08FE30E94F2
:1007A00025048093000181111BC00E941D0480E478
:1007B0000E94FB0380930001811112C08CE00E9413
:1007C00025048093000181110BC00E9425048093B1
:1007D0000001811105C08FE30E9425048093000170
:1007E0000E941D048091000108951092B9008AE0D2
:1007F0008093B800089594EA9093BC009091BC0057
:1008000097FFFCCF9091B900987F983021F09031FC
:1008100011F081E008958093BB0084E88093BC00D0
:100820008091BC0087FFFCCF8091B900887F883120
:1008300011F0803471F780E0089584E98093BC0062
:100840008091BC0084FDFCCF08958093BB0084E8B8
:100850008093BC008091BC0087FFFCCF9091B900D1
:10086000987F81E0983209F480E0089584E88093CD
:10087000BC008091BC0087FFFCCF8091BB00089535
:1008800080910001811115C080E40E94FB038093D8
:10089000000181110CC082E10E94250480930001B7
:1008A000811105C08FEF0E942504809300010E94F2
:1008B0001D0484B1807F84B985B1807F85B98AB1F8
:1008C000837F8AB98BB1837F8BB93E984698089510
:1008D0000E94A603809300010E94400480B38C70A4
:1008E00080BB81B3836F81BBA6E3B1E0E4E4F1E0B8
:1008F0008EE08E0F11921D928E13FCCF0C949003FC
:10090000BF92CF92DF92EF92FF920F931F93CF93FC
:10091000DF9380910001882379F0809135018F5F0A
:1009200080933501811108C00E94A60380930001C5
:10093000811102C00E94380306E311E0C0E0D0E05C
:10094000DD24D39482E0C82EEE24E394F12CC7304A
:10095000D10500F580910001811164C080E40E94FE
:10096000FB0380930001811112C082E10E942504E3
:100970008093000181110BC0C7010C2E01C0880FAC
:100980000A94EAF780950E942504809300010E9452
:100990001D0448C0CA30A1F028F4C83059F0C9304D
:1009A00061F005C0CC3089F070F0CD3089F0209A2C
:1009B000289810C0219A29980DC0229A2A980AC016
:1009C000239A2B9807C0529A01C0539A5B9802C091
:1009D0003E9A469890EA9A95F1F79FB1799902C0AC
:1009E00082E001C080E091709D25982B7C9902C027
:1009F00084E001C080E0892B7D9902C038E001C00D
:100A000030E0832B7E9902C020E101C020E0822BE0
:100A10009FB19095991F9927991F9295990F907E54
:100A2000892B0FC080910001811149C080E40E9490
:100A3000FB0380930001882379F1B12C0E941D04EF
:100A40008B2DF8019081981719F08083C0920101D5
:100A50000E94400421960F5F1F4FCE30D10509F050
:100A600076CF80910101882361F18150809301014B
:100A7000882339F08FE99FE00197F1F700C000006B
:100A800020C0A4E4B1E0E6E3F1E0CF01825F919100
:100A90009D938E13FCCF15C083E10E9425048093A3
:100AA00000018111CACF81E40E94FB038093000101
:100AB0008111C3CF0E943604B82EB094BFCF80E01E
:100AC000C0CF0E94360381E0DF91CF911F910F913B
:100AD000FF90EF90DF90CF90BF900895E82FF0E067
:100AE000EC5BFE4F808108950895089596E0799F0C
:100AF000F001112494E5899FE00DF11D1124E60F0A
:100B0000F11DEE0FFF1FE851FF4F8591949108955D
:100B1000880F991FFC01E05AF04085919491089547
:100B2000880F991FFC01E052FF4F85919491089521
:100B30000F931F93CF93DF93EC018115904350F5F2
:100B4000C11580E2D80708F0B3C0CB3BD10590F4C3
:100B5000C83AD10508F05AC0C53AD10508F04BC0D3
:100B6000C430D10508F0BBC1219709F0B5C101E03F
:100B700010E0F5C1CF3FD10511F008F0B0C1C03F82
:100B8000D10508F092C0CE01805E9109089708F463
:100B9000A6C1A2C1C11591E5D907A8F4C23020E5CC
:100BA000D20708F09EC0C11580E5D80709F485C0BA
:100BB00008F091C0C11520E4D20708F08DC1DD27EF
:100BC0008E01106CCCC1C11580E8D80758F4C1154E
:100BD00090E7D90708F07CC1C11520E6D20708F4D8
:100BE00022C17AC1C11580E9D80708F075C1DF704C
:100BF0008E01106AB4C1C53AD10509F472C1C63A72
:100C0000D10509F071C102E810E4A9C1C83AD105C3
:100C100009F46DC1C93AD10509F46CC1CA3AD105CC
:100C200009F46BC1CB3AD10509F46AC1CC3AD105BC
:100C300009F469C1CD3AD10509F468C1C03BD105B9
:100C400009F467C1CE3AD10509F466C1CF3AD1059E
:100C500009F465C1C13BD10509F464C1C23BD105AA
:100C600009F463C1C33BD10509F462C1C43BD1059A
:100C700009F461C1C53BD10509F460C1C63BD1058A
:100C800009F45FC1C73BD10509F45EC1C83BD1057A
:100C900009F45DC1C93BD10509F45CC1CA3BD1056A
:100CA00009F45BC100E014E45AC18E01106557C11C
:100CB000CE019F700E94900553C10E94EA149FEFDD
:100CC00024E38CE0915020408040E1F700C0000018
:100CD0000E94251C44C18091CD0181608093CD018B
:100CE0003EC10E94CE1D811102C00E94B41D0E940F
:100CF000EB1D90E09093EE018093ED01C23090E502
:100D0000D90721F48091ED01816086C0C43020E5CF
:100D1000D20721F48091ED0182607EC0C63080E56B
:100D2000D80721F48091ED01846076C0C83090E549
:100D3000D90719F48091ED0127C0CA3020E5D20708
:100D400021F48091ED01806167C0CC3080E5D80747
:100D500021F48091ED0180625FC0CE3090E5D9072B
:100D600021F48091ED01806457C0C03120E5D207A5
:100D700021F48091ED0180684FC0C23180E5D80731
:100D800029F48091ED018460886046C0C33090E50D
:100D9000D90721F48091ED018E7F3EC0C53020E55A
:100DA000D20721F48091ED018D7F36C0C73080E5F8
:100DB000D80721F48091ED018B7F2EC0C93090E5DA
:100DC000D90719F48091ED0126C0CB3020E5D20778
:100DD00021F48091ED018F7E1FC0CD3080E5D807D2
:100DE00021F48091ED018F7D17C0CF3090E5D907B8
:100DF00021F48091ED018F7B0FC0C13120E5D20736
:100E000021F48091ED018F7707C0C331D04531F4D3
:100E10008091ED018B7F877F8093ED018091ED01C3
:100E20000E94EF1D9CC08D2F99278F7099278130CC
:100E30009105D9F49E012370332702C0880F991FB2
:100E40002A95E2F79C688E0144E0000F111F4A9535
:100E5000E1F700271370802B912B53E0CC0FDD1F9F
:100E60005A95E1F7C076DD272FC08230910531F425
:100E7000DC2FCC278E01016F106A71C08330910581
:100E800069F4CE018370992701E010E002C0000FE1
:100E9000111F8A95E2F7C8019C680FC0049709F0FA
:100EA0005EC0CE018370992701E010E002C0000F00
:100EB000111F8A95E2F7C8019A6823E0CC0FDD1F65
:100EC0002A95E1F7C07ED7708C010C2B1D2B47C0F3
:100ED000DF708E01106243C000E010E040C08E0160
:100EE0003EC001E810E43BC003E810E438C002EE65
:100EF00014E435C009EE14E432C00AEE14E42FC045
:100F000005EB14E42CC006EB14E429C007EB14E451
:100F100026C00CEC14E423C00DEC14E420C003E85C
:100F200015E41DC00AE815E41AC002E915E417C06B
:100F300004E915E414C001E216E411C003E216E46A
:100F40000EC004E216E40BC005E216E408C006E297
:100F500016E405C007E216E402C00AE216E4C8017E
:100F6000DF91CF911F910F91089596E0799FF00145
:100F7000112494E5899FE00DF11D1124E60FF11D68
:100F8000EE0FFF1FE851FF4F85919491803E910530
:100F9000E0F4803C910558F58133910509F46FC068
:100FA00048F48932910509F463C08A32910509F445
:100FB0006DC072C089339105E9F082389105D1F096
:100FC0008533910509F44DC067C0833E910581F1D9
:100FD00038F4803E9105B9F0823E9105D9F05CC0AD
:100FE000863E910561F1873E9105A1F155C00E94B1
:100FF000880508952091ED0120FD02C021FF4CC01D
:1010000080EE90E049C08091ED0180FFF9CF89E347
:1010100090E042C08091ED0182FF0EC08091ED0111
:1010200084FF03C080E090E037C083EE90E034C0DE
:101030008091ED0182FFF2CF82EE90E02DC0809191
:10104000ED0183FF0BC08091ED0184FDEBCF87EEB6
:1010500090E022C08091ED0183FFF5CF86EE90E015
:101060001BC08091ED0185FF07C089E290E014C0AC
:101070008091ED0185FFF9CF85E390E00DC080916F
:10108000ED0186FF07C08AE290E006C08091ED0185
:1010900086FFF9CF81E390E00E94980508950895B6
:1010A0000C944F08809162010895CF93DF9300D094
:1010B0001F92CDB7DEB79C018091E401843019F511
:1010C00093E099833B832A839093E9008FEF90917B
:1010D000E800815095FD06C095ED9A95F1F7000066
:1010E0008111F5CF8091E80085FF0DC040E050E010
:1010F00063E070E0CE0101960E94C20A8091E80090
:101100008E778093E8000F900F900F90DF91CF9132
:101110000895CF93DF9300D01F92CDB7DEB7209113
:10112000E401243021F522E029839B838A8383E034
:101130008093E9008FEF9091E800815095FD06C003
:1011400095ED9A95F1F700008111F5CF8091E800B7
:1011500085FF0DC040E050E063E070E0CE010196F5
:101160000E94C20A8091E8008E778093E8000F9079
:101170000F900F90DF91CF9108952091E4012430DA
:10118000F1F422E02093E9002FEF3091E8002150A4
:1011900035FD06C035ED3A95F1F700002111F5CF88
:1011A0002091E80025FF0BC040E050E065E070E0D2
:1011B0000E94C20A8091E8008E778093E80008952B
:1011C000CF93DF93EC019091E401943009F046C095
:1011D00080910C018823D9F080910D018823B9F00A
:1011E0009093E9008FEF9091E800815095FD06C043
:1011F00095E19A95F1F700008111F5CF8091E80013
:1012000085FF2CC040E050E060E170E017C081E055
:101210008093E9008FEF9091E800815095FD06C022
:1012200095ED9A95F1F700008111F5CF8091E800D6
:1012300085FF14C040E050E068E070E0CE010E94FD
:10124000C20A8091E8008E778093E80080E1FE0179
:10125000A2E5B1E001900D928A95E1F7DF91CF917F
:1012600008958091E301811109C00E94570C0E94EA
:10127000B40C8091E20084608093E20008951092A3
:10128000E301089508950C945D220E94BB1B0E9407
:1012900063220E945A0F0C94500842E061EC81E0F6
:1012A0000E94D10B42E061EC82E00E94D10B42E04F
:1012B00061EC83E00E94D10B42E161EC84E00C948C
:1012C000D10B8091E601833009F455C030F48130B0
:1012D00071F0823009F48EC008958A3009F47AC022
:1012E0008B3009F460C0893009F09CC020C0809127
:1012F000E501813A09F096C08091E800877F8093EC
:10130000E8008091E9019091EA01892B21F460E1E4
:1013100082E591E003C060E080E090E070E00E9430
:101320000D0B8091E8008B778093E8000895809101
:10133000E501813209F076C08091E9019091EA01DE
:10134000009719F0039709F06DC08091E800877F3E
:101350008093E8008091E80082FD05C08091E4015F
:101360008111F8CF5FC08091F1008093620180917C
:10137000E8008B7753C08091E501813A09F052C0B3
:101380008091E9019091EA01892B09F04BC080918D
:10139000E800877F8093E8008091E80080FFFCCF21
:1013A00080910C0136C08091E5018132D9F58091A0
:1013B000E9019091EA01892BA9F58091E800877FE6
:1013C0008093E8000E94060C8091E70180930C0155
:1013D0000C94EA148091E501813221F58091E800B6
:1013E000877F8093E8000E94060C8091E80180933B
:1013F000630108958091E501813AA1F48091E800AC
:10140000877F8093E8008091E80080FFFCCF809187
:1014100063018093F1008091E8008E778093E8006B
:101420000C94060C089584B7877F84BF0FB6F89498
:10143000A8958091600088618093600010926000A0
:101440000FBE90E080E80FB6F8948093610090930F
:1014500061000FBE0E94A90F0E94570C0E94B40C9D
:101460008091E20084608093E20078940E943A0FB9
:101470000E94AB0F82E091E00E94550F0E944B2228
:101480008091E401853069F40E94791B8091E2012A
:101490008823B1F30E94A71B882391F30E94AC0A12
:1014A000EFCF0E94B10FECCF292F33272330310526
:1014B000C9F064F42130310581F02230310509F0A2
:1014C00043C08DE690E02CEB33E042C02132310581
:1014D000F1F02232310541F137C082E190E029E29A
:1014E00034E036C099278130910541F08230910572
:1014F00041F0892B49F5E8EBF3E005C0E0EAF3E0C1
:1015000002C0E8E8F3E0849190E09F0121C06430DC
:10151000D8F4E62FF0E0EE0FFF1FEE5DFE4F2081C6
:10152000318189E090E014C0643070F470E0FB0118
:10153000EE0FFF1FE65EFE4F20813181FB01EA5E68
:10154000FE4F808190E004C080E090E020E030E039
:10155000FA0131832083089580E189BD82E189BD4C
:1015600009B400FEFDCF8091D8008F7D8093D80014
:101570008091E00082608093E0008091E00081FD36
:10158000FCCF0895CF92DF92EF92FF920F931F93BB
:10159000CF93DF93EC018B016A010E94250C81112E
:1015A00033C0C114D10439F0F60180819181081B48
:1015B000190BC80FD91FE12CF12C0115110519F1D8
:1015C0008091E80085FD16C08091E8008E778093B9
:1015D000E800C114D10449F0F60180819181E80E40
:1015E000F91EF182E08285E00FC00E94250C88235D
:1015F00021F30AC089918093F10001501109FFEF96
:10160000EF1AFF0ADACF80E0DF91CF911F910F919F
:10161000FF90EF90DF90CF9008952091EB013091F3
:10162000EC012617370748F06115710539F4209150
:10163000E8002E772093E80001C0B90140E0611571
:101640007105A9F12091E401222309F443C025305A
:1016500009F442C02091E80023FD40C02091E80039
:1016600022FD32C02091E80020FFE9CF4091F30035
:101670002091F20030E0342BFC01CF01611571059F
:1016800059F02830310540F481918093F100615088
:1016900071092F5F3F4FF1CF41E02830310509F04C
:1016A00040E02091E8002E772093E800C8CF411158
:1016B000C9CF0AC08091E401882361F0853061F0D0
:1016C0008091E80083FD0AC08091E80082FFF2CF9C
:1016D00080E0089582E0089583E0089581E0089510
:1016E0002091EB013091EC012617370748F0611586
:1016F000710539F42091E8002E772093E80001C0AD
:10170000B901FC0120E06115710591F18091E401BE
:10171000882309F440C0853009F43FC08091E80077
:1017200083FD3DC08091E80082FD2FC08091E800DC
:1017300080FFE9CF2091F3008091F20090E0922B9E
:101740006115710559F08830910540F4249120937A
:10175000F1003196615071090196F2CF21E00897AE
:1017600009F020E08091E8008E778093E800CBCFED
:101770002111CCCF0AC08091E401882361F085302B
:1017800061F08091E80083FD0AC08091E80082FF4B
:10179000F2CF80E0089582E0089583E0089581E02B
:1017A0000895982F973058F59093E900981739F0DD
:1017B0007091EC002091ED005091F00003C0242FB7
:1017C000762F50E021FF19C03091EB003E7F30931F
:1017D000EB003091ED003D7F3093ED003091EB0058
:1017E00031603093EB007093EC002093ED00509348
:1017F000F0002091EE0027FF07C09F5FD3CF8F70CE
:101800008093E90081E0089580E008958091E501EA
:1018100087FF11C08091E80082FD05C08091E4013E
:101820008111F8CF11C08091E8008B770BC08091B7
:10183000E401882349F08091E80080FFF8CF80918F
:10184000E8008E778093E80008952091E4003091BD
:10185000E50095E64091EC00842F817040FF22C0A6
:101860008091E80080FD1CC08091E401882391F004
:10187000853091F08091EB0085FD10C04091E4002F
:101880005091E5004217530729F39A01915011F73F
:1018900084E0089582E0089583E0089581E008954A
:1018A00080E008954091E80042FFDECF08950E9455
:1018B000C50C0E94CD0CE0EEF0E080818160808359
:1018C000E8EDF0E080818F77808319BCA7EDB0E070
:1018D0008C918E7F8C9380818F7E80831092E30128
:1018E00008950F931F93CF93DF930E94C50C0E941E
:1018F000CD0CC8EDD0E088818F778883888180689F
:10190000888388818F7D888319BC1092E4011092AE
:10191000E0011092E2011092E10100EE10E0F80106
:1019200080818B7F808388818160888342E060E052
:1019300080E00E94D10BE1EEF0E080818E7F808319
:10194000E2EEF0E080818160808380818860808326
:10195000F80180818E7F8083888180618883DF9118
:10196000CF911F910F910895E8EDF0E080818F7E77
:101970008083E7EDF0E080818160808384E082BF36
:1019800081E08093E3010C94710CE8EDF0E080813C
:101990008E7F80831092E20008951092DA001092F8
:1019A000E10008951F920F920FB60F9211242F930A
:1019B0003F934F935F936F937F938F939F93AF93D7
:1019C000BF93EF93FF938091E10082FF0BC0809162
:1019D000E20082FF07C08091E1008B7F8093E100ED
:1019E0000E94390F8091DA0080FF1FC08091D800DB
:1019F00080FF1BC08091DA008E7F8093DA00809197
:101A0000D90080FF0DC080E189BD82E189BD09B4A4
:101A100000FEFDCF81E08093E4010E94310905C002
:101A200019BC1092E4010E943F098091E10080FFFF
:101A300019C08091E20080FF15C08091E2008E7F86
:101A40008093E2008091E20080618093E2008091C7
:101A5000D80080628093D80019BC85E08093E401AF
:101A60000E9443098091E10084FF30C08091E20030
:101A700084FF2CC080E189BD82E189BD09B400FEEC
:101A8000FDCF8091D8008F7D8093D8008091E100B8
:101A90008F7E8093E1008091E2008F7E8093E20050
:101AA0008091E20081608093E2008091E0018823D0
:101AB00011F084E007C08091E30087FD02C081E05F
:101AC00001C083E08093E4010E9445098091E10018
:101AD00083FF29C08091E20083FF25C08091E1004F
:101AE000877F8093E10082E08093E4011092E0011F
:101AF0008091E1008E7F8093E1008091E2008E7FF3
:101B00008093E2008091E20080618093E20042E0F5
:101B100060E080E00E94D10B8091F00088608093AB
:101B2000F0000E944209FF91EF91BF91AF919F9108
:101B30008F917F916F915F914F913F912F910F9076
:101B40000FBE0F901F9018951F920F920FB60F9215
:101B500011242F933F934F935F936F937F938F93B2
:101B60009F93AF93BF93CF93DF93EF93FF93C09176
:101B7000E900CF708091EC00D82FD17080FDD0E8C3
:101B80001092E9008091F000877F8093F0007894B4
:101B90000E94E80D1092E9008091F0008860809327
:101BA000F000CD2BCF70C093E900FF91EF91DF9152
:101BB000CF91BF91AF919F918F917F916F915F91E5
:101BC0004F913F912F910F900FBE0F901F9018953E
:101BD0001F93CF93DF93CDB7DEB7AA970FB6F894D4
:101BE000DEBF0FBECDBFE5EEF1E088E08E0F909135
:101BF000F10091938E13FBCF0E9461098091E80060
:101C000083FF1FC18091E5019091E601492F50E0CB
:101C10004A30510508F015C1FA01EA5AFF4F0C94F9
:101C2000F423803881F0823809F00BC18091E901FA
:101C30008F708093E9008091EB0085FB882780F905
:101C40001092E90006C08091E1019091E2019111AA
:101C500082609091E800977F9093E8008093F10074
:101C60001092F100C8C0282F2D7F09F0EAC0882308
:101C700019F0823061F0E5C08091E701813009F010
:101C8000E0C0933009F080E08093E2012BC08091A6
:101C9000E701811127C08091E9018F7009F4D1C05B
:101CA0008093E9002091EB0020FF1CC0933021F4C9
:101CB0008091EB00806214C09091EB009061909352
:101CC000EB0021E030E0A90102C0440F551F8A95C6
:101CD000E2F74093EA001092EA008091EB008860FE
:101CE0008093EB001092E9008091E800877F86C026
:101CF0008111A7C01091E7011F778091E3008078E0
:101D0000812B8093E3008091E800877F8093E80037
:101D10000E94060C8091E80080FFFCCF8091E300D8
:101D200080688093E300111102C082E001C083E06B
:101D30008093E40186C08058823008F082C0809190
:101D4000E7019091E8018C3D53E0950779F583E038
:101D50008A838AE289834FB7F894DE01139620E0E4
:101D60003EE051E2E32FF0E050935700E49120FF72
:101D700003C0E295EF703F5FEF708E2F90E0EA3086
:101D800010F0C79601C0C0968D939D932F5F2431AC
:101D900049F74FBF8091E800877F8093E8006AE2AF
:101DA00070E0CE0101960E940D0B14C0AE014F5F92
:101DB0005F4F6091E9010E94540ABC01892B09F42C
:101DC00040C09091E800977F9093E80089819A81C4
:101DD0000E94700B8091E8008B778093E80031C0FF
:101DE000803879F58091E800877F8093E8008091C2
:101DF000E0018093F1008091E8008E778093E80005
:101E00000E94060C1EC081111CC09091E701923007
:101E1000C0F48091E800877F8093E8009093E00110
:101E20000E94060C8091E001811106C08091E300C0
:101E300087FD02C081E001C084E08093E4010E943C
:101E40004D098091E80083FF0AC08091E800877FF8
:101E50008093E8008091EB0080628093EB00AA966B
:101E60000FB6F894DEBF0FBECDBFDF91CF911F91AB
:101E700008950895CF938091E4018823A1F0C09143
:101E8000E900CF709091EC00892F817090FD80E87F
:101E9000C82B1092E9008091E80083FD0E94E80DB4
:101EA000CF70C093E900CF9108959093690180931A
:101EB00068010895E0916801F0916901309721F07F
:101EC0000190F081E02D099480E00895E09168018F
:101ED000F0916901309721F00280F381E02D09949F
:101EE0000895E0916801F0916901309721F0048034
:101EF000F581E02D099408952091660130916701E4
:101F00008217930771F09093670180936601E091C7
:101F10006801F0916901309721F00680F781E02D8A
:101F20000994089520916401309165018217930707
:101F300071F09093650180936401E0916801F091E4
:101F40006901309721F00084F185E02D099408950E
:101F500008950C94A80F0E94C11B0E9468040C9461
:101F6000871CCF92DF92EF92FF920F931F93CF9334
:101F7000DF93CDB7DEB72B970FB6F894DEBF0FBE59
:101F8000CDBF0E9480048BE6C82E81E0D82E00E0F1
:101F900010E0E02E802F0E946E05F60141916F0146
:101FA000F42EF826B1F40F5F1F4F0E30110589F79C
:101FB0008FEF89838A831B820E94CA1B8160782FDE
:101FC0009D838C8349815A816B818D810E9454103D
:101FD00040C09091CD0191FF04C08B870E94740591
:101FE0008B8520E030E04F2D50E0922FBA01022E79
:101FF00002C0759567950A94E2F760FF24C02E83AE
:10200000EF8221E030E0690102C0CC0CDD1C9A9522
:10201000E2F790E08C219D21892B09F420E02887AC
:102020000E94CA1B8160782F9A8789874E815F81C1
:1020300068858A850E945410F801E559FE4F808119
:10204000C826C08206C02F5F3F4F2630310569F693
:10205000AACF0E946E1F10916A010E945A0F181792
:10206000A1F00E945A0F80936A012B960FB6F89444
:10207000DEBF0FBECDBFDF91CF911F910F91FF90BB
:10208000EF90DF90CF900C9450082B960FB6F894F9
:10209000DEBF0FBECDBFDF91CF911F910F91FF909B
:1020A000EF90DF90CF900895CF93DF93CDB7DEB759
:1020B0002B970FB6F894DEBF0FBECDBF4F83588766
:1020C00069877A878B87DE01119686E0FD01119280
:1020D0008A95E9F785E0FE01379601900D928A9581
:1020E000E1F749815A816B817C818D819E810E94BB
:1020F00084172B960FB6F894DEBF0FBECDBFDF91CD
:10210000CF9108950895CF93882309F4C2C0C82FB2
:10211000823859F40E945A0F81FDBBC089E30E94A6
:102120002D1A0E94FA1A89E30CC0833879F40E94B0
:102130005A0F80FDAEC083E50E942D1A0E94FA1A44
:1021400083E50E946F1ACF910C94FA1A843859F4DF
:102150000E945A0F82FD9DC087E40E942D1A0E94A2
:10216000FA1A87E4EECF8CEF8C0F813A48F48C2F6B
:102170000E94B02181118DC08C2F0E942D1AE3CFB7
:1021800080E28C0F883048F4C77081E001C0880F6E
:10219000CA95EAF70E94B31AD6CF8BE58C0F83302D
:1021A00078F4C53A29F0C63A31F083E890E005C0EA
:1021B00081E890E002C082E890E0CF910C947C0F1F
:1021C00088E58C0F833108F064C0C83A39F1C93A08
:1021D00041F1CA3A49F1CB3A51F1CC3A59F1CD3AF1
:1021E00061F1C03B69F1CE3A71F1CF3A79F1C13B6F
:1021F00081F1C23B89F1C33B91F1C43B99F1C53BED
:10220000A1F1C63BA9F1C73BB1F1C83BB9F1C93B4C
:10221000C1F1CA3BC9F180E090E038C082EE90E0A5
:1022200035C089EE90E032C08AEE90E02FC085EB99
:1022300090E02CC086EB90E029C087EB90E026C0B0
:102240008CEC90E023C08DEC90E020C083E891E01E
:102250001DC08AE891E01AC082E991E017C084E9C4
:1022600091E014C081E292E011C083E292E00EC0DE
:1022700084E292E00BC085E292E008C086E292E040
:1022800005C087E292E002C08AE292E0CF910C940E
:10229000920FCF910895882309F44BC0823859F4E6
:1022A0000E945A0F81FF45C089E30E942D1A0E94A7
:1022B000FA1A89E30CC0833871F40E945A0F80FF28
:1022C00038C083E50E942D1A0E94FA1A83E50E9405
:1022D0006F1A0C94FA1A843859F40E945A0F82FF2C
:1022E00028C087E40E942D1A0E94FA1A87E4EFCFD3
:1022F0009CEF980F913A58F390E2980F983050F471
:10230000877091E001C0990F8A95EAF7892F0E94A2
:10231000B91ADFCF9BE5980F933020F480E090E06E
:102320000C947C0F885A833120F480E090E00C9468
:10233000920F0895882321F00E94B31A0C94FA1A80
:102340000895882321F00E94B91A0C94FA1A08956E
:10235000BF92CF92DF92EF92FF920F931F93CF9392
:10236000DF9300D000D000D0CDB7DEB725E0FC0170
:10237000DE01119601900D922A95E1F7FC01D080C3
:1023800011810281258122952F7043815481452B33
:1023900009F4FCC21F3F21F4FFEFDF1609F4F6C277
:1023A0007C012E830E948210D9821A8369817A81EE
:1023B000802F0E94291A182FB92E0E94DE190E9420
:1023C000A5182E81002319F00E94D01A2E81EB2D22
:1023D000E295EF70F0E0E05AFF4F0C94F4238B2D60
:1023E000807F9B2D9F70F92E882319F0F29480EF47
:1023F000F822002389F0FF2009F475C280E2810FE2
:10240000883020F48F2D0E94B31A03C08F2D0E94B4
:10241000C31A0E94FA1A67C2812F0E944B11FF2033
:1024200009F4B4C2105E8F2D183018F40E94B91A46
:1024300002C00E94C91A26960FB6F894DEBF0FBEDE
:10244000CDBFDF91CF911F910F91FF90EF90DF9063
:10245000CF90BF900C94FA1A3B2D307F8B2D8F704C
:10246000303211F08295807F112319F0113021F163
:102470002CC00023B9F0222309F4A0C1213009F0B7
:102480009DC126960FB6F894DEBF0FBECDBFDF917B
:10249000CF911F910F91FF90EF90DF90CF90BF9061
:1024A0000C94E31A222319F0213009F46FC28E83B1
:1024B0000E94E61A8E8196C1002321F0223008F096
:1024C00065C27CC1211162C28DC1002321F022238B
:1024D00009F474C108C2222309F484C119C22B2D46
:1024E00026952695237030E02115310521F0213005
:1024F0003105D1F04BC2002321F0812F9B2D937029
:1025000002C080E090E026960FB6F894DEBF0FBEC2
:10251000CDBFDF91CF911F910F91FF90EF90DF9092
:10252000CF90BF900C947C0F002321F0812F9B2D26
:10253000937002C080E090E026960FB6F894DEBF5C
:102540000FBECDBFDF91CF911F910F91FF90EF9004
:10255000DF90CF90BF900C94920F812F002319F041
:102560000E94761E02C00E94DE1E26960FB6F894C8
:10257000DEBF0FBECDBFDF91CF911F910F91FF90B6
:10258000EF90DF90CF90BF900C94631F8B2D8370E2
:1025900009F07BC00111FAC1812F82958695877061
:1025A000880F880F912F9F70C92ED12CE12CF12C10
:1025B000082E04C0CC0CDD1CEE1CFF1C0A94D2F7C4
:1025C00014FF12C04FE050E060E070E004C0440F20
:1025D000551F661F771F8A95D2F7CB01BA01609508
:1025E00070958095909503C060E070E0CB012B2D35
:1025F000269526952370422F50E042305105D9F0A0
:102600004330510569F16C297D298E299F2941307C
:10261000510551F126960FB6F894DEBF0FBECDBF1F
:10262000DF91CF911F910F91FF90EF90DF90CF90AE
:10263000BF900C94CC186C297D298E299F29269651
:102640000FB6F894DEBF0FBECDBFDF91CF911F91C3
:102650000F91FF90EF90DF90CF90BF900C94E8180F
:102660000E94CC18C701B60126960FB6F894DEBFBB
:102670000FBECDBFDF91CF911F910F91FF90EF90D3
:10268000DF90CF90BF900C94B018002319F08B2DE1
:10269000817001C08695882309F478C1812F8295C5
:1026A00086958770880F880F912F9F70C92ED12C27
:1026B000E12CF12C082E04C0CC0CDD1CEE1CFF1C00
:1026C0000A94D2F714FF12C04FE050E060E070E0CF
:1026D00004C0440F551F661F771F8A95D2F7CB01A0
:1026E000BA01609570958095909503C060E070E0A8
:1026F000CB012B2D269526952370422F50E042309A
:102700005105D9F04330510569F16C297D298E2995
:102710009F294130510551F126960FB6F894DEBF3E
:102720000FBECDBFDF91CF911F910F91FF90EF9022
:10273000DF90CF90BF900C94A6196C297D298E292B
:102740009F2926960FB6F894DEBF0FBECDBFDF914E
:10275000CF911F910F91FF90EF90DF90CF90BF909E
:102760000C94C2190E94A619C701B60126960FB68D
:10277000F894DEBF0FBECDBFDF91CF911F910F91B7
:10278000FF90EF90DF90CF90BF900C948A19103F8C
:10279000D1F118F4103E50F4A1C0123F09F463C007
:1027A00008F44CC0133F09F473C098C01F708B2D00
:1027B0008F710023A1F00E942319812F26960FB656
:1027C000F894DEBF0FBECDBFDF91CF911F910F9167
:1027D000FF90EF90DF90CF90BF900C949A110E94E1
:1027E0004419812F26960FB6F894DEBF0FBECDBFD9
:1027F000DF91CF911F910F91FF90EF90DF90CF90DD
:10280000BF900C94A1110023A9F02111BFC08B2D02
:102810008F7126960FB6F894DEBF0FBECDBFDF9145
:10282000CF911F910F91FF90EF90DF90CF90BF90CD
:102830000C946919223008F0A9C0E9CF0023A9F04F
:102840008B2D8F7126960FB6F894DEBF0FBECDBFCD
:10285000DF91CF911F910F91FF90EF90DF90CF907C
:10286000BF900C942319002359F38B2D8F7126965A
:102870000FB6F894DEBF0FBECDBFDF91CF911F9191
:102880000F91FF90EF90DF90CF90BF900C94441980
:10289000002399F08B2D8F7126960FB6F894DEBF2A
:1028A0000FBECDBFDF91CF911F910F91FF90EF90A1
:1028B000DF90CF90BF900C940E1926960FB6F89427
:1028C000DEBF0FBECDBFDF91CF911F910F91FF9063
:1028D000EF90DF90CF90BF900C9404190023A9F0E3
:1028E000222309F4ADCF812F26960FB6F894DEBFD0
:1028F0000FBECDBFDF91CF911F910F91FF90EF9051
:10290000DF90CF90BF900C948310222309F4ADCFB9
:10291000812F26960FB6F894DEBF0FBECDBFDF9194
:10292000CF911F910F91FF90EF90DF90CF90BF90CC
:102930000C944B114B2D4F70612FC7010E94040363
:1029400026960FB6F894DEBF0FBECDBFDF91CF91B4
:102950001F910F91FF90EF90DF90CF90BF900C945C
:1029600028184B2D4F70612FC70126960FB6F8948B
:10297000DEBF0FBECDBFDF91CF911F910F91FF90B2
:10298000EF90DF90CF90BF900C94750526960FB610
:10299000F894DEBF0FBECDBFDF91CF911F910F9195
:1029A000FF90EF90DF90CF90BF9008950E94D01AD3
:1029B0000E94E01A0E94A51A0E94FA1A0E9413208F
:1029C0000E94631F80E090E00E947C0F80E090E016
:1029D0000C94920F0E94C01A0C94D6140E941E1AD6
:1029E000292F22952F7030E02C3031054CF42A30FD
:1029F00031056CF4225031092230310588F407C0CA
:102A00002C30310549F02F30310531F009C0803EBE
:102A100048F0803F29F406C093FB882780F9089589
:102A200080E0089581E00895CF93DF9300D000D037
:102A30001F92CDB7DEB70F900F900F900F900F90B1
:102A4000DF91CF910895CF93DF9300D000D000D0D5
:102A5000CDB7DEB726960FB6F894DEBF0FBECDBF5A
:102A6000DF91CF9108951F93CF93DF93C0917901A8
:102A700016E080917A01C81799F0D0E01C9FF00110
:102A80001D9FF00D1124E558FE4F40815181628158
:102A90007381848195810E9423152196C770E9CFA7
:102AA000DF91CF911F9108954091AB015091AC01FE
:102AB0006091AD017091AE018091AF019091B00134
:102AC0000C9423158091B00182958F7009F054C049
:102AD0008091AD01882309F44FC080917901A091C4
:102AE0007A016091AB017091AC014091AE015091BF
:102AF000AF01B6E08A1709F43FC090E041155105D7
:102B0000C1F17F3F11F46F3FA1F1B89FF001B99F70
:102B1000F00D1124E558FE4F218172132AC0208147
:102B2000621327C02281211124C0238134812417FC
:102B3000350710F421503109241B350B283C310591
:102B4000C0F42091B0012F7020612093B00126E0E5
:102B5000289FF001299FF00D1124E058FE4F80813D
:102B60008F70806180838BEA91E00E94A8110C94A1
:102B7000331501968770BECF0895CF92DF92EF9202
:102B8000FF920F931F93CF93DF93CDB7DEB762977A
:102B90000FB6F894DEBF0FBECDBF8C0185E0F80103
:102BA000DE011D9601900D928A95E1F7D8014C91B6
:102BB00011965C91119712966C9112971396CD9085
:102BC000DC9014973091AB017091AC018091AE0113
:102BD0009091AF01009709F46BC17F3F19F43F3F1B
:102BE00009F466C1E090AD01EE2009F4C0C0209167
:102BF000B001C816D90628F0F601E81BF90BCF0181
:102C000004C0809590958C0D9D1DFF24F394883C05
:102C1000910578F0F12C207F09F0C6C07C2DD98A6F
:102C2000C88A89890E9414158BEA91E00E94A81134
:102C3000B1C0822F807F09F046C0751314C03413D1
:102C400012C0611110C02F7020612093B0010E944A
:102C500054158BEA91E00E94A8118091B001D8012F
:102C600015968C932EC0CD2819F15F3F11F44F3F7C
:102C7000F9F0F62E61111CC08091790120917A0142
:102C800036E0821709F45AC090E0389FF001399F6E
:102C9000F00D1124E558FE4F7181571306C0708165
:102CA000471303C07281711103C001968770E9CF89
:102CB000F62E662309F418C18091B00181608093DB
:102CC000B001F12C11C1751308C0341306C0611195
:102CD00004C08091B001D801C3C04D875E878D8547
:102CE0009E856A8B0E94EE146A898823E1F166232F
:102CF000D1F12091B001822F82958F7090E00297E0
:102D000074F08091AB019091AC0198878F83198604
:102D1000DB86CA862C87CE0107960E94A81186E022
:102D2000F801ABEAB1E001900D928A95E1F70E94BB
:102D300062150E945415FF24F394D6C04D875E8718
:102D40008D859E850E941E1A292F22952F7030E0B6
:102D5000223031050CF0BCC09F7009F0B6C0805E17
:102D6000883008F4C1C0C8010E94A811E4CFC81679
:102D7000D90608F453C0F601E81BF90BCF01883CD3
:102D8000910508F450C0F12C7C2DD98AC88A898914
:102D90000E941415EBEAF1E086E0DF011D928A95AE
:102DA000E9F70E945415A0C0751314C0341312C063
:102DB000611110C08091B001F8018583C8010E94A3
:102DC000A81186E0EBEAF1E0DF011D928A95E9F7B0
:102DD000FE2C8AC04D875E878D859E856A8B0E94FA
:102DE000EE146A89882309F4BECF662309F4BBCFA9
:102DF0002091B001822F82958F7090E002970CF4A1
:102E00008ECF8091AB019091AC019A8389831B8214
:102E1000DD82CC822E83CE0101967FCF8095909566
:102E20008C0D9D1DACCFF62E662309F49CCF751337
:102E30002EC034132CC02091B00120FD1FC0822F62
:102E400082958F70D9F0D80115962C9315978F30F5
:102E500049F08F5F982F9295907F822F8F70892BEA
:102E600015968C93C8010E94A81186E0F801ABEA80
:102E7000B1E001900D928A95E1F793CF86E0F801D9
:102E8000ABEAB1E001900D928A95E1F72DC04D8734
:102E90005E878D859E850E94EE14811140CF8091C2
:102EA000B00181608093B001C8010E94A8111CC0CC
:102EB000662309F458CF4D875E878D859E850E94D5
:102EC000EE14882309F44FCF2ACF811148CF0CC0CC
:102ED000243031050CF047CF9F7009F440CFF80142
:102EE0009581907F09F03BCF8F2D62960FB6F894B5
:102EF000DEBF0FBECDBFDF91CF911F910F91FF902D
:102F0000EF90DF90CF9008951F93CF93DF93CDB7CD
:102F1000DEB72C970FB6F894DEBF0FBECDBF4F8340
:102F2000588769877A878B879C87CE0107960E948E
:102F3000BD15882369F08F8198852A853B85232BD1
:102F4000F1F19F3F09F063C08F3F09F060C037C0C7
:102F500086E0FE013796DE01119601900D928A956A
:102F6000E1F76F817885EA85FB85309741F17F3FF6
:102F700011F46F3F21F120917A0130E0C9010196EF
:102F8000877099274091790150E08417950709F4DB
:102F900047C069837A83FD83EC8396E0929FD001DA
:102FA000939FB00D1124A558BE4FFE01319601909C
:102FB0000D929A95E1F780937A010E94331516E0FD
:102FC0008091790190917A018917C1F1189FC00110
:102FD000112485589E4F0E94BD15882379F1E091F8
:102FE00079011E9FF0011124E558FE4F4081518167
:102FF00062817381848195810E942315809179017A
:1030000090E001968770992780937901D9CF4F81FD
:10301000588569857A858B859C850E942315CFCF3D
:103020000E94EA1410927A0110927901EBEAF1E021
:1030300086E0DF011D928A95E9F7C1CF2C960FB685
:10304000F894DEBF0FBECDBFDF91CF911F910895E1
:10305000EF92FF920F931F93CF93DF938C01892BF5
:1030600009F46CC0F12CEE24E394E8012196F801F8
:103070008491843740F4843008F051C0813081F06D
:10308000823019F15BC0853709F444C0A8F19CE790
:10309000980F903708F052C08F770E944B1141C0B3
:1030A0000E5F1F4FFE01C49180E28C0F883048F400
:1030B000C7708E2D01C0880FCA95EAF70E94D31AF7
:1030C00014C08C2F0E9483102DC00E5F1F4FFE0175
:1030D000C49180E28C0F883058F4C7708E2D01C0E7
:1030E000880FCA95EAF70E94D91A0E94FA1A1AC0E4
:1030F0008C2F0E944B1116C00E5F1F4FFE01C49112
:10310000CC2381F08FE99FE00197F1F700C0000028
:10311000C150F6CF0E5F1F4FFE01F49003C00E9416
:1031200083108E018F2D882309F49FCFEFE9FFE0F4
:103130003197F1F700C000008150F5CFDF91CF91BA
:103140001F910F91FF90EF90089508956093B5013E
:103150007093B6018093B7019093B8010C94D61484
:103160000F931F930091B5011091B6012091B70103
:103170003091B801DC01CB01802B912BA22BB32B1A
:103180008093B5019093B601A093B701B093B801B5
:103190001F910F910C94D6140F931F930091B501BA
:1031A0001091B6012091B7013091B801DC01CB013B
:1031B00080239123A223B3238093B5019093B6017A
:1031C000A093B701B093B8011F910F910C94D6143E
:1031D0000F931F930091B5011091B6012091B70193
:1031E0003091B801DC01CB0180279127A227B327BA
:1031F0008093B5019093B601A093B701B093B80145
:103200001F910F910C94D6141092B1011092B2013B
:103210001092B3011092B4010C94D61441E050E026
:1032200060E070E004C0440F551F661F771F8A9549
:10323000D2F74093B1015093B2016093B301709300
:10324000B4010C94D61441E050E060E070E004C09A
:10325000440F551F661F771F8A95D2F78091B101E1
:103260009091B201A091B301B091B401482B592BB8
:103270006A2B7B2B4093B1015093B2016093B30151
:103280007093B4010C94D61441E050E060E070E01B
:1032900004C0440F551F661F771F8A95D2F74095CB
:1032A0005095609570958091B1019091B201A09177
:1032B000B301B091B401482359236A237B2340937F
:1032C000B1015093B2016093B3017093B4010C94B7
:1032D000D61441E050E060E070E004C0440F551F98
:1032E000661F771F8A95D2F78091B1019091B20144
:1032F000A091B301B091B401482759276A277B27D1
:103300004093B1015093B2016093B3017093B40143
:103310000C94D6140F931F930091B1011091B20138
:103320002091B3013091B401DC01CB01802B912BB2
:10333000A22BB32B8093B1019093B201A093B30160
:10334000B093B4011F910F910C94D6140F931F9357
:103350000091B1011091B2012091B3013091B401FB
:10336000DC01CB0180239123A223B3238093B101FD
:103370009093B201A093B301B093B4011F910F9148
:103380000C94D6140F931F930091B1011091B201C8
:103390002091B3013091B401DC01CB01802791274A
:1033A000A227B3278093B1019093B201A093B301F8
:1033B000B093B4011F910F910C94D6140895CF923D
:1033C000DF92EF92FF920F931F93CF93DF938C01C5
:1033D000C090B501D090B601E090B701F090B8016F
:1033E0008091B1019091B201A091B301B091B4016B
:1033F000C82AD92AEA2AFB2ACFE1D0E0D701C601A0
:103400000C2E04C0B695A795979587950A94D2F788
:1034100080FF06C0B8018C2F0E94B507019721F4E8
:10342000219760F780E001C08C2FDF91CF911F9131
:103430000F91FF90EF90DF90CF900895CF93DF939F
:10344000EC010E94DF19BE010E94B507DF91CF9108
:103450000895CB010E941E1A089590910C019923A2
:1034600021F090910D01911109C020910E01309130
:103470000F01F90132969FEF40E01FC0982F9695FB
:10348000969596959F3050F5E0910E01F0910F01C1
:10349000E90FF11D877021E030E0A90102C0440F5F
:1034A000551F8A95E2F7CA019181892B818308957E
:1034B0009F3F39F04F5F4E3041F051915813F8CF94
:1034C0000DC05111F7CF942FF5CF9F3F39F0F9017F
:1034D000E90FF11D97FDFA95828308950895909163
:1034E0000C01992321F090910D01911109C02091B7
:1034F0000E0130910F01F9013296205F3F4F1FC03E
:10350000982F9695969596959F30F0F4E0910E0140
:10351000F0910F01E90FF11D877021E030E0A90162
:1035200002C0440F551F8A95E2F7CA018095918128
:103530008923818308953196E217F30729F090815A
:103540009813F9CF1082F7CF089581E090E0E091D1
:103550000E01F0910F01E80FF91F108201968031E2
:103560009105A9F708959091CC01892B8093CC0106
:10357000089580959091CC0189238093CC01089582
:103580001092CC0108959091CB01892B8093CB01AF
:10359000089580959091CB0189238093CB01089564
:1035A0001092CB0108959091CA01892B8093CA0192
:1035B000089580959091CA0189238093CA01089546
:1035C0001092CA0108958093B90108951092B9012B
:1035D000089580910E0190910F01FC0131969C019C
:1035E000205F3F4F80E0919191118F5FE217F307C9
:1035F000D1F70895E0910E01F0910F018091CC0177
:103600008083E0910E01F0910F0190818091CB01B8
:10361000892B8083E0910E01F0910F0190818091C0
:10362000CA01892B80838091B901882361F0E091E0
:103630000E01F0910F019081892B80830E94E91A7D
:1036400081111092B90180910E0190910F010C949B
:10365000660FCF92DF92EF92FF926C01EE24FF246F
:10366000C114D104E104F10421F0C701B60120E145
:1036700001C020E0C72ED82EE92EFF24C114D104AA
:10368000E104F10419F0285FC701B6016B017C0168
:1036900054E0F694E794D794C7945A95D1F7C1149F
:1036A000D104E104F10419F02C5FC701B6016B01EC
:1036B0007C0142E0F694E794D794C7944A95D1F7F9
:1036C000C114D104E104F10419F02E5FC701B60161
:1036D000DC01CB01B695A79597958795892B8A2B09
:1036E0008B2B09F02F5F822FFF90EF90DF90CF9010
:1036F00008958091E401843039F11092CE0120E4E4
:1037000088E190E00FB6F894A895809360000FBE12
:103710002093600080E00E94500883B7817F84601E
:1037200083BF83B7816083BF7894889583B78E7F8A
:1037300083BF0FB6F894A89580916000886180934C
:103740006000109260000FBE089508950895CF9311
:103750000E94A51B0E9480040E94A61BC0E08C2F23
:103760000E946E05811104C0CF5FCE30C1F701C049
:1037700081E0CF9108950E94EA140E945A0F0C94A0
:10378000500882E084BD93E095BD9AEF97BD809389
:103790006E0008952FB7F8948091CF019091D001D9
:1037A000A091D101B091D2012FBF0895CF92DF92A5
:1037B000EF92FF920F931F932FB7F8944091CF0190
:1037C0005091D0016091D1017091D2012FBF6A0157
:1037D0007B01EE24FF248C0120E030E0C016D106EE
:1037E000E206F30610F4415051099A01281B390BE7
:1037F000C9011F910F91FF90EF90DF90CF90089536
:103800001F920F920FB60F9211248F939F93AF9335
:10381000BF938091CF019091D001A091D101B0913F
:10382000D2010196A11DB11D8093CF019093D001CB
:10383000A093D101B093D201BF91AF919F918F918D
:103840000F900FBE0F901F9018950E94570CF89480
:103850002FEF87EA91E6215080409040E1F700C0C9
:10386000000087E090EBDC018093EE019093EF0184
:10387000A093F001B093F1019CE088E10FB6F894B9
:10388000A895809360000FBE90936000FFCFEF92E9
:10389000FF920F931F93CF93DF93D82FC0E08C2F0D
:1038A0000E946E0500E010E0E82EF12CC701002E0A
:1038B00002C0959587950A94E2F780FD06C00F5FD8
:1038C0001F4F0630110591F709C0602F7C2F80E053
:1038D0000E947605D813F3CF81E004C0CF5FCE30CD
:1038E000F1F680E0DF91CF911F910F91FF90EF9063
:1038F0000895CF93C82F8CE20E94471C882321F0A3
:103900008C2FCF910C94471C80E0CF910895CF93DA
:103910000E94CE1D811102C00E94B41DC5E6C15097
:1039200049F00E9480048FE39CE90197F1F700C001
:103930000000F5CF89E20E94791C811113C18AE24F
:103940000E94791C81110E94B41D85E00E94791C9F
:1039500081110E94251C0E94D91D8093CD0187E012
:103960000E94791C8823A9F18BE10E94791C88238D
:1039700051F08091CD0181FB222720F991E092271F
:1039800090FB81F90EC08EE00E94791C882361F0C3
:103990008091CD0182FB222720F991E0922790FBB4
:1039A00082F98093CD0115C080E10E94791C90912D
:1039B000CD01882341F093FB222720F981E0822763
:1039C00080FB93F904C0892F809580FB90F9909338
:1039D000CD018091CD010E94DD1D0E94EB1D8093E1
:1039E000ED0180EE0E94791C882341F08091ED0169
:1039F000982F909590FB80F98093ED0189E30E94C8
:103A0000791C882359F08091ED0181FB222720F950
:103A100091E0922790FB81F98093ED0182EE0E9464
:103A2000791C882359F08091ED0182FB222720F92F
:103A300091E0922790FB82F98093ED0186EE0E943F
:103A4000791C882359F08091ED0183FB222720F90E
:103A500091E0922790FB83F98093ED0183EE0E9421
:103A6000791C882359F08091ED0184FB222720F9ED
:103A700091E0922790FB84F98093ED0185E30E9409
:103A8000791C882359F08091ED0185FB222720F9CC
:103A900091E0922790FB85F98093ED0181E30E94EC
:103AA000791C882359F08091ED0186FB222720F9AB
:103AB00091E0922790FB86F98093ED0181E10E94CD
:103AC000791C882359F08091ED0187FB222720F98A
:103AD00091E0922790FB87F98093ED018091ED01B1
:103AE0000E94EF1D8091ED0187FB882780F980936C
:103AF0000D0187E20E94791CC82F8EE10E94791C7B
:103B00008111C2608FE10E94791C8111C46080E242
:103B10000E94791C8111C86081E20E94791C811188
:103B2000C06182E20E94791C8111C06283E20E941E
:103B3000791C8111C06484E20E94791C882311F0F1
:103B4000C06802C0CC2329F08C2F0E94E61D6C2F88
:103B500003C00E94E21D682F70E080E090E0CF91EA
:103B60000C94A618CF9108956DEE7EEF80E090E062
:103B70000E942E2460E082E090E00E941C2460E01D
:103B800083E090E00E941C2460E084E090E00E94CA
:103B90001C2460E085E090E00C941C2480E090E020
:103BA0000E94162421E08D3E9E4F09F020E0822FD6
:103BB000089582E090E00C940E24682F82E090E05B
:103BC0000C941C2483E090E00C940E24682F83E076
:103BD00090E00C941C2484E090E00C940E24682F58
:103BE00084E090E00C941C248091D50180FF0BC0F0
:103BF0006091130185E0689FB00111247595679568
:103C0000759567952BC081FF09C06091130185E010
:103C1000689FB00111247595679520C082FF07C089
:103C20006091130185E0689FB001112417C0909145
:103C3000D6019923D1F060911201961788F720914F
:103C4000130185E0289F90011124929FA001939F6A
:103C5000500D112470E0CA010E94E0236038710504
:103C600040F46115710539F002C065E070E0862FFF
:103C700008958FE7089581E008958091D50180FF30
:103C800008C06091110170E075956795759567950D
:103C900021C081FF06C06091110170E075956795A4
:103CA00019C082FF04C06091110170E010C09091B2
:103CB000D6019923C1F0609110019617A0F7809169
:103CC0001101899FC001112470E00E94E023603837
:103CD000710528F46115710521F0862F08958FE78D
:103CE000089581E0089561E070E0F4CF803F21F411
:103CF0000E94F41D819504C0813F29F40E94F41DA7
:103D00008093D9010895823F21F40E94F41D81958A
:103D100004C0833F29F40E94F41D8093D8010895C4
:103D2000893F19F40E943D1E05C08A3F31F40E946C
:103D30003D1E81958093DA0108958B3F21F40E9406
:103D40003D1E819504C08C3F29F40E943D1E809346
:103D5000DB010895843F21F48091D701816017C071
:103D6000853F21F48091D701826011C0863F21F404
:103D70008091D70184600BC0873F21F48091D701E7
:103D8000886005C0883F31F48091D70180618093BD
:103D9000D70108958D3F21F48091D50181600BC03A
:103DA0008E3F21F48091D501826005C08F3F29F4B8
:103DB0008091D50184608093D5010895803F39F4C6
:103DC0008091D90187FF6CC01092D90169C0813FF1
:103DD00029F48091D9011816BCF362C09091D801E2
:103DE000823F29F497FF5CC01092D80159C0833FED
:103DF00019F41916CCF354C0893F41F48091DA01CB
:103E000018160CF04DC01092DA014AC08A3F29F40E
:103E10008091DA0187FF44C0F6CF8B3F39F480915F
:103E2000DB0187FF3DC01092DB013AC08C3F29F4D3
:103E30008091DB011816BCF333C0843F21F48091DC
:103E4000D7018E7F17C0853F21F48091D7018D7FE8
:103E500011C0863F21F48091D7018B7F0BC0873F33
:103E600021F48091D701877F05C0883F31F480918C
:103E7000D7018F7E8093D70113C08D3F21F48091AD
:103E8000D5018E7F0BC08E3F21F48091D5018D7FAF
:103E900005C08F3F29F48091D5018B7F8093D50198
:103EA0008091D80181110EC08091D90181110AC081
:103EB0008091DA01811106C08091DB01811102C07D
:103EC0001092D601089587ED91E00E94710F0E9433
:103ED000CA1B9093D4018093D30108951F93CF936D
:103EE000DF938091D3019091D4010E94D61BAC0145
:103EF0009091D601992321F02091140130E006C061
:103F0000209115018AE0289F900111244217530740
:103F100008F485C08091D801C091D901D091DA010F
:103F20001091DB01811107C0C11175C0D11173C09F
:103F3000111171C074C09F3F19F09F5F9093D6011B
:103F4000181624F40E94F41D8093D8018091D801A2
:103F500087FF05C00E94F41D81958093D8011C162F
:103F600024F40E94F41D8093D9018091D90187FF28
:103F700005C00E94F41D81958093D9016091D801FC
:103F8000662331F1C091D901CC2311F1062E000C2A
:103F9000770B880B990B0E94E72223E333E343E37B
:103FA0005FE30E944B230E94AF226093D8016C2FE5
:103FB000CC0F770B880B990B0E94E72223E333E3A6
:103FC00043E35FE30E944B230E94AF226093D90139
:103FD0001D1624F40E943D1E8093DA018091DA01BF
:103FE00087FF05C00E943D1E81958093DA0111165E
:103FF00024F40E943D1E8093DB018091DB0187FF4A
:1040000005C00E943D1E81958093DB01DF91CF9119
:104010001F910C94631F9F3F09F08FCF97CFDF91C3
:10402000CF911F910895E7EDF1E085E0DF011D924A
:104030008A95E9F71092D6011092D5010895833040
:1040400081F128F4813059F08230D1F00895853023
:1040500009F449C0B8F1863009F456C0089580913A
:104060001501262F30E0280F311D2F3F310524F494
:10407000680F6093150108958FEF809315010895DF
:1040800080911401262F30E0280F311D2F3F31057C
:1040900024F4680F6093140108958FEF8093140146
:1040A000089580911301262F30E0280F311D2F3FF6
:1040B000310524F4680F6093130108958FEF809306
:1040C0001301089580911201262F30E0280F311D31
:1040D0002F3F310524F4680F6093120108958FEF8C
:1040E00080931201089580911101262F30E0280F4E
:1040F000311D2F3F310524F4680F6093110108959D
:104100008FEF80931101089580911001262F30E0E8
:10411000280F311D2F3F310524F4680F60931001E3
:1041200008958FEF809310010895833011F128F4E2
:10413000813049F0823091F00895853081F120F18D
:104140008630C1F1089580911501681720F4861B0F
:10415000809315010895109215010895809114011E
:10416000681720F4861B809314010895109214019F
:10417000089580911301681720F4861B8093130122
:10418000089510921301089580911201681720F488
:10419000861B809312010895109212010895809158
:1041A0001101681720F4861B809311010895109265
:1041B0001101089580911001681720F4861B8093E7
:1041C000100108951092100108950F931F938D31DF
:1041D00009F46BC008F03FC08E3009F47FC0C0F412
:1041E000873009F469C068F4863009F0B1C0809165
:1041F000CD01817F8E7F8093CD0181E08093DD01B1
:10420000A8C0883009F4A2C08B3009F49FC0A0C0B8
:10421000863109F49BC078F4803109F472C0813191
:1042200009F096C00E94EA1490910D0181E089275F
:1042300080930D018BC0893109F488C08B3109F05E
:1042400087C08091CD0181FB222720F991E0922740
:1042500090FB81F94CC0853309F470C048F4873273
:1042600009F46CC008F459C0893209F467C070C001
:10427000833438F48A3308F04EC0883309F466C0BA
:1042800067C0833409F45AC0883409F061C00E94C1
:10429000EA140FEF13ED20E3015010402040E1F746
:1042A00000C000000E94251C51C00E9469220E948B
:1042B0005A0F0E9450084AC09091CD01892F8095D5
:1042C000817080FB90F929F0966098609093CD0101
:1042D00040C0997F977F9093CD0138C08091CD01E8
:1042E00082FB222720F991E0922790FB82F98093AC
:1042F000CD01992359F18091CD0181608093CD0149
:1043000025C08091CD0183FB222720F991E09227DF
:1043100090FB83F9ECCF895301C08D5141E050E00F
:1043200060E070E08A019B0104C0000F111F221F92
:10433000331F8A95D2F7C901B80104C061E070E06B
:1043400080E090E00E94A6180E94EA1481E001C07B
:1043500080E01F910F91089580E0089580E0089516
:10436000CF93C82F8091DD01813079F018F0823031
:10437000E9F187C0E0910E01F0910F018081813158
:1043800069F0823209F07FC009C0E0910E01F0911E
:104390000F018081813111F0823261F48C2F0E94F3
:1043A000AC21811104C08C2F0E94E5201DC081E04A
:1043B00090E01AC08C2F0E94AE21811114C0C4312C
:1043C00079F048F4CB3079F0C03109F060C082E078
:1043D0008093DD0108C0C93219F0C83321F057C0FD
:1043E0001092DD0154C081E0817053C0C93289F15F
:1043F00018F5C43171F1A8F4C73009F046C08AE05D
:104400008093150194E19093140193E0909313012C
:104410008093120188E08093110188E2809310015B
:1044200034C0CE51C63088F5EC2FF0E0E65DFE4F8B
:1044300080818093DC0129C0CE34E9F020F4CB34B4
:1044400021F56AE013C0C13579F0C235F1F461E0BD
:104450000DC08091DC01882319F01092DC0115C099
:1044600081E08093DD0115C061E006C08091DC0130
:104470000E941F200AC06AE08091DC010E94952002
:1044800004C01092DD0180E004C081E002C080E041
:10449000ABCFCF910895E1E8F0E080818860808320
:1044A0008081816080838FB7F89493E09093890036
:1044B00090ED909388008FBF0895EFE6F0E0808143
:1044C000826080830895EFE6F0E080818D7F8083B5
:1044D0000895EFE6F0E0908182E0892780830895D7
:1044E0001F920F920FB60F9211242F933F934F9369
:1044F0005F936F937F938F939F93AF93BF93EF934C
:10450000FF938091DE019091DF0101969093DF018E
:104510008093DE01811103C082E00E945008E09187
:10452000DF01E695E695F0E0EA5CFA4FE4918091D0
:10453000DE018E1303C080E00E945008FF91EF91CE
:10454000BF91AF919F918F917F916F915F914F91AB
:104550003F912F910F900FBE0F901F9018950E94C2
:10456000B6226894B1110C94452308950E942A2321
:1045700088F09F5798F0B92F9927B751B0F0E1F024
:10458000660F771F881F991F1AF0BA95C9F714C0D4
:10459000B13091F00E944423B1E008950C9444237B
:1045A000672F782F8827B85F39F0B93FCCF386950D
:1045B00077956795B395D9F73EF49095809570956A
:1045C00061957F4F8F4F9F4F0895E89409C097FBE7
:1045D0003EF490958095709561957F4F8F4F9F4FDA
:1045E0009923A9F0F92F96E9BB279395F69587951E
:1045F00077956795B795F111F8CFFAF4BB0F11F4E1
:1046000060FF1BC06F5F7F4F8F4F9F4F16C0882387
:1046100011F096E911C0772321F09EE8872F762FBD
:1046200005C0662371F096E8862F70E060E02AF0FE
:104630009A95660F771F881FDAF7880F96958795EA
:1046400097F9089557FD9058440F551F59F05F3F53
:1046500071F04795880F97FB991F61F09F3F79F0A4
:1046600087950895121613061406551FF2CF469526
:10467000F1DF08C0161617061806991FF1CF8695A8
:104680007105610508940895E894BB27662777278C
:10469000CB0197F908950E945E230C94CF230E94CA
:1046A000C12338F00E94C82320F0952311F00C9408
:1046B000B8230C94BE2311240C9445230E9422237A
:1046C00070F3959FC1F3950F50E0551F629FF00165
:1046D000729FBB27F00DB11D639FAA27F00DB11D7E
:1046E000AA1F649F6627B00DA11D661F829F222707
:1046F000B00DA11D621F739FB00DA11D621F839F8E
:10470000A00D611D221F749F3327A00D611D231F63
:10471000849F600D211D822F762F6A2F11249F57B1
:1047200050409AF0F1F088234AF0EE0FFF1FBB1FB4
:10473000661F771F881F91505040A9F79E3F510573
:1047400080F00C94B8230C9445235F3FE4F3983E2B
:10475000D4F3869577956795B795F795E7959F5F1D
:10476000C1F7FE2B880F911D9695879597F90895AF
:1047700097F99F6780E870E060E008959FEF80EC14
:10478000089500240A9416161706180609060895B7
:1047900000240A9412161306140605060895092E1D
:1047A0000394000C11F4882352F0BB0F40F4BF2B8C
:1047B00011F460FF04C06F5F7F4F8F4F9F4F0895CC
:1047C00097FB072E16F4009407D077FD09D00E94BE
:1047D000FA2307FC05D03EF4909581959F4F0895EC
:1047E000709561957F4F0895EE0FFF1F0590F4912E
:1047F000E02D0994AA1BBB1B51E107C0AA1FBB1FD8
:10480000A617B70710F0A61BB70B881F991F5A955C
:10481000A9F780959095BC01CD010895F999FECF37
:1048200092BD81BDF89A992780B50895A8E1B0E0BE
:1048300042E050E00C943624262FF999FECF92BD29
:1048400081BDF89A019700B4021639F01FBA20BD55
:104850000FB6F894FA9AF99A0FBE08950196272F89
:104860000E941D240C941C24DC01CB01FC01F9994D
:10487000FECF06C0F2BDE1BDF89A319600B40D92AC
:0C48800041505040B8F70895F894FFCF65
:10488C0020025208E008BD08890855080101BA0148
:10489C0028080A03140A3F4D3639F704AA04740495
:1048AC003B04CE03E70300041904010203040506CC
:0448BC0007080900E0
:00000001FF
